:0400000002003F3289
:01000B0032C2
:0100130032BA
:01001B0032B2
:0100230032AA
:01002B0032A2
:01003300329A
:03003B000219D3D4
:0300BF000200C27A
:0500C2001200D780FED2
:0E00C700E582900001F0900001E0FAF582025F
:0200D5000E56C5
:0700D700121E70120E2C1224
:0900DE0001A11201147582021245
:0200E70001B85E
:0E00E90090012C1201177582021201B9AA8231
:0B00F7007B00C002C0037468C0E0740E
:0C0102001FC0E07480C0E0121019E581FD
:06010E0024FBF58180D501
:041F680025640A00E2
:030114000202F9EB
:0E011700AA83E582900011F0A3EAF090001197
:0E012500E0FAA3E0FB90001DEAF0A3EBF090DF
:08013300000275F0001202FF4A
:0C013B0090000275F00012036250F522E3
:06008F00E478FFF6D8FD45
:08004C007909E94400601B7A08
:0500540001901FD278AD
:03005900E175A0AE
:0A005C0000E493F2A308B8000205C7
:08006600A0D9F4DAF275A0FF45
:0E0147009000641203D612057EE5828583F0D7
:09015500900013F0A3E5F0F02284
:0D015E00900013E0FAA3E0FB8A828B83126D
:09016B000587120520758290122F
:0D01740005324020758240120532400F9088
:0C0181000017E0FAF5821205324003027C
:02018D00052A41
:09018F0012052A75820202194AC8
:0901980012052A75820102194AC0
:0E01A1009000641203D612057EE5828583F07D
:0901AF00900015F0A3E5F0F02228
:0101B8002224
:0E01B900E582900018F0900015E0FAA3E0FB3C
:0E01C7008A828B8312058712052075829012A2
:0C01D50005324028900018E0FAF5821274
:0B01E1000532402512052075829112A6
:0701EC0005324011C20012B0
:0E01F3000571AA82C00212052AD0028A822259
:0902010012052A75820112194A46
:09020A0012052A75820202194A4C
:0E021300E582900019F0900019E0FAF58212D1
:0E02210001B9AA827B008A057C00EA2CFAEB68
:06022F003D8A82F58322E6
:0E023500AAF0AB83E58290001AF0A3EBF0A3D1
:0E024300EAF0900015E0FAA3E0FB8A828B83BC
:0A0251001205871205207582901235
:09025B0005325005740124FF2254
:0D0264007582041205325005740124FF223A
:0E027100120520758291120532500574012489
:02027F00FF225C
:06028100D200120571908D
:0C028700001AE0FAA3E0FBA3E0FC7D00FD
:0E029300901F6CE493FEC3ED9E50547F001E3E
:0402A100BEFF011F7C
:0E02A5008D007900E8B50608E9B507047E0073
:0202B3008002C7
:0202B5007E01C8
:0C02B700EE24FF9200ED2AFEE43BFF8CD9
:0E02C30000C002C003C004C005C006C007C0D2
:0E02D10000120571A982D000D007D006D0051A
:0E02DF00D004D003D0028E828F8388F0E91203
:0502ED000AA20D80A132
:0702F20012052AE424FF229B
:011F6C000470
:011F6D000172
:0602F9001219FF0205A826
:0E02FF00AAF0AB83E58290001FF0A3EBF0A302
:0E030D00EAF090001FE0FAA3E0FBA3E0FC740E
:09031B000B2AF508E43BF5098CFE
:0C0324000A1219ABAD82AE83AFF0F89066
:0E033000001DE0F9A3E0FAE4FBFCE92DFDEA74
:0C033E003EFEEB3FFFEC38F8850882859E
:07034A000983850AF0ED12A2
:0A0351000AA2A3EE120AA2A3EF1203
:07035B000AA2A3E8020AA2B6
:0A036200C00E85810EC082C083C06A
:0E036C00F0E5812407F5811219ABAD82AE8356
:0C037A00AFF0FAE50E2404F8A60508A672
:0C0386000608A60708A602A80E08740BC3
:0E03920026FBE40836FC0886028B828C838AE8
:0C03A000F0121E79FBA3121E79FCA312C0
:0903AC001E79FAA3121E79FDE589
:0C03B5000E2404F8C3EB96EC0896EA084E
:0C03C10096ED08965006740124FF80039E
:0303CD00E424FF26
:0603D000850E81D00E2213
:0E03D600AA83E582900022F0A3EAF0D297D22B
:0E03E40096120B7CE433FABA010890002574DF
:0403F20001F0800690
:0603F6009000257402F0E6
:0E03FC00900024E4F0900022E0FAA3E0FB7CE5
:01040A0000F1
:03040B00BC07002B
:05040E0040030204ABF5
:0E041300EC75F003A4FDFE901F6E93CEA39334
:0E042100FF900025E0F8790090004FE8F0A36E
:0E042F00E9F08E828F83C002C003C004C005B6
:0E043D00C000C001120ABBAE82AF83D001D056
:0E044B0000D005D004D003D002C3EA9EEB9F80
:0A0459004047ED246EFDE4341FFE61
:0E0463008D828E83A3A3E493FFA2E292DFEFCB
:0E047100A2E192D9EF1392D88D828E83E4938C
:0E047F00FDA3E493FE90004FE8F0A3E9F08D9A
:0E048D00828E83120ABBE5828583F0900022E6
:07049B00F0A3E5F0F0800979
:0904A2000C900024ECF002040BA4
:0E04AB00900024E0FABA0757EA14900024F0FB
:0C04B900900024E0FA75F003A4246EFA11
:0C04C500E4341FFB8A828B83A3A3E49322
:0E04D100FCA2E292DFECA2E192D9EC1392D8E9
:0E04DF008A828B83E493FAA3E493FB900025BA
:0E04ED00E0FC90004FF0A3E4F08A828B8312B3
:0E04FB000ABBE5828583F0900022F0A3E5F0B5
:01050900F001
:0E050A00C2DBC2DCC2DDC2DAD2DE900022E02B
:08051800FAA3E08A82F58322B8
:04052000C2DBD2DD8B
:0605240030DBFDC2DD2208
:04052A00D2DCC2DB82
:04052E0020DCFD22AE
:0E053200E582900026F0900026E0F5DAC2DBAC
:0A05400030DBFDAAD9BA18028019B9
:05054A00BA2002801838
:05054F00BA2802800F34
:05055400BA3002800E28
:05055900BA400280051C
:05055E00BA480B800407
:04056300E424FF226B
:05056700740124FF22D5
:05056C00740124FF22D0
:06057100A20092DAC2DBD9
:0705770030DBFD85DA822272
:09057E00AAD87B008A828B83223B
:0E058700AA83E582900027F0A3EAF0900027F7
:0E059500E0FAA3E0FBEA3392DFEAA2E192D99A
:0505A300EA1392D822CA
:0E1F6E00660206330105E60003C00002A4006F
:071F7C0001900000260004A3
:0200B900C20182
:0405A80030010122FB
:0C05AC009000E1E4F0A3F0A3F0D20122E3
:0E05B800AAF0AB83E58290002DF0A3EBF0A338
:0E05C600EAF090002DE0FAA3E0FBA3E0FC8A2F
:0E05D400828B838CF0E4120AA274042AFDE4E8
:0E05E2003BFE8C07900029E0F8A3E0F98D8223
:0E05F0008E838FF0E8120AA2A3E9120AA27409
:0E05FE00062AFDE43BFE8C0790002BE0F8A3DC
:0E060C00E0F98D828E838FF0E8120AA2A3E936
:0B061A00120AA274012AF514E43BF55B
:04062500158C16908A
:0C06290000E1E0F8A3E0F9A3E0FD851477
:09063500828515838516F0E81298
:0A063E000AA2A3E9120AA2A3ED121A
:0E0648000AA29000E1EAF0A3EBF0A3ECF0228E
:0E065600AAF0AB83E582900037F0A3EBF0A38F
:0E066400EAF0900037E0FAA3E0FBA3E0FC8A86
:0E067200828B838CF07401120AA274042AFD9C
:0E068000E43BFE8C07900030E0F8A3E0F98D1B
:0E068E00828E838FF0E8120AA2A3E9120AA25C
:0E069C0074062AFDE43BFE8C07900032E0F865
:0E06AA00A3E0F98D828E838FF0E8120AA2A3DE
:0C06B800E9120AA274082AF514E43BF5CC
:0406C400158C1690EB
:0C06C8000034E0F8A3E0F9A3E0FD851485
:0906D400828515838516F0E812F9
:0A06DD000AA2A3E9120AA2A3ED127B
:0A06E7000AA274012AF514E43BF5A1
:0406F100158C1690BE
:0C06F50000E1E0F8A3E0F9A3E0FD8514AB
:09070100828515838516F0E812CB
:0A070A000AA2A3E9120AA2A3ED124D
:0E0714000AA29000E1EAF0A3EBF0A3ECF022C1
:0E072200AAF0AB83E58290003AF0A3EBF0A3BF
:0E073000EAF0900040E4F0A3F0A3F09000E1A6
:0E073E00E0FAA3E0FBA3E0FC90003DEAF0A38C
:0C074C00EBF0A3ECF090003AE0F514A3F1
:07075800E0F515A3E0F51622
:0E075F0090003DE0FDA3E0FEA3E0FFBD00071B
:07076D00BE0004BF000122E1
:0A077400EDB5140AEEB51506EFB559
:04077E0016028003DC
:030782000207F774
:0E078500900040E0FCA3E0FBA3E0FABC0030D3
:0E079300BB002DBA002A74012DF8E43EF98F48
:0D07A10002888289838AF0121E79F8A31263
:0907AE001E79F9A3121E79FA90DC
:0C07B70000E1E8F0A3E9F0A3EAF08034D0
:0C07C30074012CF8E43BF90DBD00010EA0
:0E07CF008D828E838FF0121E79FDA3121E798B
:0E07DD00FEA3121E79FF888289838AF0ED1236
:0A07EB000AA2A3EE120AA2A3EF1265
:0207F5000AA256
:0E07F70090003DE0FAA3E0FBA3E0FC90004080
:0D080500EAF0A3EBF0A3ECF00ABA00010B3F
:0E0812008A828B838CF0121E79FAA3121E7953
:0E082000FBA3121E79FC90003DEAF0A3EBF062
:06082E00A3ECF002075FDD
:0E083400AAF0AB83E582900043F0A3EBF0A3A3
:0E084200EAF0900043E0FAA3E0FBA3E0FC8A9A
:08085000828B838CF002072269
:0E0858009000E1E0FAA3E0FBA3E0FCBA000888
:06086600BB0005BC00020E
:02086C0080FE0C
:05086E0012087380FB7D
:0E0873009000E1E0FAA3E0FBA3E0FC90004659
:08088100EAF0A3EBF0A3ECF098
:0E088900900046E0FAA3E0FBA3E0FCBA0007F3
:07089700BB0004BC000122BC
:0E089E008A828B838CF0121E79FDBD010280D0
:0108AC000348
:0308AD00020971CC
:0E08B00074042AFDE43BFE8C078D828E838F3C
:0E08BE00F0121E79FDA3121E79FE74082AF5B1
:0608CC000BE43BF50C8C6F
:0A08D2000DC002C003C004850B82B4
:0708DC00850C83850DF0126D
:0A08E3001E79FAA3121E79FBA3127E
:0E08ED001E79FCC002C003C004C005C0067422
:0A08FB000DC0E07409C0E0C005C0A4
:08090500068A828B838CF0222C
:0C090D00D006D005D004D003D002920226
:0C091900D004D003D0022002030209DD4C
:0E09250074062AFDE43BFE8C078D828E838FC4
:0B093300F0121E79FDA3121E79FE8554
:06093E000B82850C83858D
:080944000DF0121E79FFA31251
:0D094C001E79F8A3121E79F9C005C00674CB
:0A0959006BC0E07409C0E0C005C0E7
:08096300068F82888389F022CF
:06096B00D006D005806CEF
:0E09710074042AFDE43BFE8C078D828E838F7A
:0E097F00F0121E79FDA3121E79FEC002C00305
:0B098D00C004C005C00674A0C0E074E8
:0809980009C0E0C005C0062201
:0D09A000D006D005D004D003D002E433F51A
:0A09AD000BE50B602B74062AFAE438
:0E09B7003BFB8A828B838CF0121E79FAA3120E
:0C09C5001E79FBC002C00374D9C0E074AE
:0809D10009C0E0C002C00322CE
:0409D900D003D00275
:0E09DD00900046E0FAA3E0FBA3E0FC0ABA009B
:0209EB00010BFE
:0E09ED008A828B838CF0121E79FAA3121E7977
:0E09FB00FBA3121E79FC900046EAF0A3EBF07D
:060A0900A3ECF0020889D5
:0E0A0F00AA83E582900049F0A3EAF09000E18E
:0E0A1D00E0FAA3E0FBA3E0FC90004BEAF0A39C
:0D0A2B00EBF0A3ECF0900049E0FAA3E0FB33
:0E0A380090004BE0FCA3E0FDA3E0FEBC000834
:080A4600BD0005BE0002804D59
:0E0A4E0074062CFFE43DF88E018F82888389A8
:0E0A5C00F0121E79FFA3121E79F8EFB5020BFF
:0B0A6A00E8B503078C828D838EF0221C
:050A75000CBC00010DA6
:0E0A7A008C828D838EF0121E79FCA3121E79E1
:0E0A8800FDA3121E79FE90004BECF0A3EDF0E2
:050A9600A3EEF0809DBD
:070A9B0090000075F000223D
:031FD2000000000C
:0E0AA20020F71030F6118883A88220F507F6A1
:050AB000A8837583001E
:010AB500221E
:030AB600F280F7D4
:020AB900F02229
:080095007800E84400600A79DC
:03009D000075A04B
:0600A00000E4F309D8FCA6
:0800A60078E0E84400600C79E9
:0B00AE0001900001E4F0A3D8FCD9FA97
:0E0ABB00AA83E582900051F0A3EAF090005368
:0E0AC900E4F0A3F090004FE0FAA3E0FB7C10F5
:0C0AD700900051E0FDA3E0FE339203EE1E
:0E0AE300CD25E0CD33FE900051EDF0A3EEF0F6
:0E0AF100900053E0FDA3E0FECD25E0CD33FEE6
:0C0AFF00900053EDF0A3EEF030031290D5
:0E0B0B000053E0FDA3E0FE90005374014DF096
:030B1900A3EEF058
:0E0B1C00900053E0FDA3E0FEC3ED9AEE9B4077
:0D0B2A001D900053EDC39AF0EE9BA3F090D8
:0E0B37000051E0FDA3E0FE90005174014DF06E
:030B4500A3EEF02C
:0E0B4800DC8D900051E0FAA3E08A82F5832252
:0200BB00D2066B
:0C0B5600A2AF9204C2AF43A220A982907B
:0E0B62000055E0FA900056E0FB8A838B821269
:0C0B7000FFF0F58253A2DFA20492AF2236
:0A0B7C00200607E4A2053324FF223F
:080B8600C206900055E4F09056
:0E0B8E0000567403F0758200120B56AA82E422
:040B9C00BA80010416
:0A0BA00024FF9205E4A2053324FFB0
:010BAA002228
:0D0BAB0090000F120117758203121EF590C5
:0E0BB8000005120117758203121EF5758203E7
:0D0BC600121EF5758203121EF575822012B5
:0C0BD3001F23758201121F2375820C1273
:080BDF001F23758201021F2390
:0E0BE700E58290007AF090007AE0FA6005BA9C
:040BF500011E800E4F
:0E0BF900900079E0FA74802AFAF582021F2338
:0E0C0700900079E0FA74C02AFAF582021F23E9
:010C150022BC
:0E0C1600E58290007EF090007EE0FAC4035468
:0E0C2400F8FA74402AFAF582121F2390007B22
:0A0C3200E0FAA3E0FBA3E0FC7D085C
:0E0C3C008A828B838CF0121E79FEA3AA82ABF3
:0E0C4A00838E82C002C003C004C005121ECDFE
:0B0C5800D005D004D003D002DDDA226A
:040C63007A017B0097
:0E0C6700C3EA9402EB6480948050558A041C0A
:0A0C7500ECC454F02459FCE43400F0
:0E0C7F00FD7E008A07EBC454F0CFC4CF6FCFC8
:0B0C8D0054F0CF6FF8EF2459FFE8345B
:0C0C980000F8900086EFF0A3E8F0A374D1
:0E0CA40000F09000897410F0E4A3F08C828DB3
:0E0CB200838EF0C002C003120EFFD003D002EA
:070CC0000ABA00A30B80A09B
:0E0CC70090008E7420F090008F7410F0E4A363
:0A0CD500F090006975F000020F7541
:040CDF007A007B001C
:0E0CE300C3EA9402EB6480948050718A0490FE
:0E0CF1000079E4F08C82C002C003120BE7D041
:0E0CFF0003D0028A04EBC454F0CCC4CC6CCCFD
:090D0D0054F0CC6CFD7E007F0067
:0D0D1600C3EE9410EF648094805036EC24FE
:0A0D230059F8ED3400F9EE28F582CE
:0E0D2D00EF39F583E0F8F582C002C003C00480
:0E0D3B00C005C006C007121ECDD007D006D0DE
:0E0D490005D004D003D0020EBE00C20F80BF42
:050D57000ABA00010BC7
:030D5C00020CE3A3
:010D5F002271
:0A0D600075820C121F23120CDF90A5
:0A0D6A000057E0FA900058E0FB90FB
:0C0D74000079F08A82120BE775820D02F4
:020D80001F232F
:0D0D8200900057E0FA90005774012AF0909D
:0E0D8F000057E0FAC3648094824009120C639E
:060D9D009000577401F004
:010DA300222D
:0E0DA400E58290007FF0900057E0FAC454F012
:080DB2002459FAE43400FB901F
:0E0DBA000058E0FC2AFAE43BFB90007FE0FDCD
:0D0DC8008A828B83F090005874012CF0900B
:0E0DD5000058E0FAC3648094904008900058E3
:050DE300E4F0020D82A6
:010DE80022E8
:0E0DE900E582900080F0900080E0FABA0902E6
:020DF700801664
:050DF900BA0A028009A6
:090DFE00BA0D26900058E4F02221
:080E0700900058E4F0020D8296
:0E0E0F00758220120DA4758220120DA475822A
:0A0E1D0020120DA4758220020DA41E
:050E27008A82020DA407
:070E2C00120114120BAB9040
:090E33000057E4F0900058F09023
:0E0E3C00008E7420F090008F7420F0E4A3F07C
:0A0E4A0090005975F000120F7502B8
:020E54000D602F
:080E5600AA82120DE9020D60F1
:0E0E5E00AAF0AB83E582900081F0A3EBF0A335
:0E0E6C00EAF0900081E0FAA3E0FBA3E0FC7D39
:030E7A00007E00F7
:0E0E7D00ED2AFFEE3BF88C018F82888389F00E
:0E0E8B00121E79FF60208F82C002C003C004D7
:0E0E9900C005C006120DE9D006D005D004D069
:0A0EA70003D0020DBD00CF0E80CC79
:030EB100020D60CF
:0C0EB400E582900085F0900085E0FA9047
:090EC0000057F0900084E0FB9063
:0B0EC9000058F0900079EBF08A8202E4
:020ED4000BE72A
:0E0ED60090008E7420F090008F7420F0E4A342
:0E0EE400F090005975F000120F757582011222
:0B0EF2001F23900084E4F075820002D2
:020EFD000EB431
:011F8300104D
:011F8400025A
:0E0EFF00AAF0AB83E58290008BF0A3EBF0A38A
:0B0F0D00EAF090008BE0F517A3E0F580
:060F180018A3E0F519909A
:0C0F1E000086E0FDA3E0FEA3E0FF8517C5
:030F2A0014851813
:030F2D001585190E
:090F300016900089E0F8A3E0F935
:090F39008802890318B8FF0119B0
:0E0F4200EA4B60258D828E838FF0121E79FAA5
:0A0F5000A3AD82AE838514828515DF
:0B0F5A00838516F0EA120AA2A385822C
:060F65001485831580CE07
:070F6B0085178285188385BC
:030F720019F02251
:0E0F7500AAF0AB83E582900091F0A3EBF0A30D
:0E0F8300EAF0900091E0FAA3E0FBA3E0FC90FE
:0C0F9100008EE0FD90008FE0FEA3E0FF6A
:090F9D008E008F011EBEFF011F32
:0E0FA600E84960118A828B838CF0ED120AA25A
:070FB400A3AA82AB8380E2D7
:0E0FBB00900091E0FAA3E0FBA3E0FC8A828B99
:040FC900838CF02203
:080FCD00C00E85810EAA8212FC
:050FD50000C7D00E2250
:0E0FDA00AAF0AB83E582900095F0A3EBF0A3A4
:0E0FE800EAF0900095E0FAA3E0FBA3E0FC9095
:0E0FF6000094E0FD9000A8E4F0A3F0A3F090BA
:0E10040000ABEAF0A3EBF0A3ECF09000AEED31
:07101200F0900FCD02113236
:06101900C00E85810EE50A
:0C101F000E24FBFA9000A8E4F0A3F0A35C
:0C102B00F0E50E24FBF89000ABE6F008A6
:0D103700A3E6F008A3E6F09000AEEAF0900A
:0A1044000FCD121132AA82AB83D047
:02104E000E2270
:0C105000E5829000A4F09000A4E0FA906B
:0E105C00009AE0C0E0A3E0C0E0A3E0C0E074B2
:08106A007EC0E07410C0E090AC
:0C1072000098E0C0E0A3E0C0E08A822209
:0E107E001581158115819000A2E0FAA3E0FB18
:0C108C009000A274012AF0E43BA3F022C3
:0E109800E5829000A5F09000A5E0FA74302AE1
:0C10A600FA24C6500A74072AFA30070327
:0310B200430220D6
:0510B5008A82021050C8
:0E10BA00E5829000A6F09000A6E0FAC4540F64
:0E10C800FBF582C002121098D00253020F8A6C
:0410D60082021098EA
:0E10DA00E5829000A7F090009DE0FAA3E0FBF5
:0E10E800A3E0FCA3E0FD9000A1E0FE9000A7B5
:0410F600E0FF78207F
:0E10FA00EE2EFEED235401F94206EA2AFAEB2F
:0E11080033FBEC33FCED33FDC3EE9F4007EEEE
:06111600C39FFE4302012D
:0E111C00D8DC90009DEAF0A3EBF0A3ECF0A36A
:08112A00EDF09000A1EEF022AF
:0E113200AA83E5829000AFF0A3EAF09000AF30
:0E114000E0FAA3E0FB900098EAF0A3EBF09039
:0E114E0000A8E0FAA3E0FBA3E0FC90009AEA00
:0E115C00F0A3EBF0A3ECF09000A2E4F0A3F0FF
:0E116A009000ABE0FAA3E0FBA3E0FC8A828BCE
:0E117800838CF0121E79FD9000AB74012AF0FA
:0D118600E43BA3F0A3ECF0ED700302185958
:05119300BD25028003F0
:03119800021851E9
:05119B00C208C209C2F8
:0411A0000AC20BC2B2
:0411A4000CC20DC2AA
:0411A8000EC20F90D4
:0911AC0000B1E4F09000B2F090F3
:0E11B50000B374FFF09000ABE0FAA3E0FBA3E0
:0211C300E0FC4E
:0E11C5008A828B838CF0121E79FEA3AA82AB65
:0D11D300839000ABEAF0A3EBF0A3ECF090EA
:0D11E00000B5EEF0BE25088E821210500200
:0211ED00116A85
:0511EF008E07BF300077
:0E11F40040498E07EF24C640429000B3E0FF52
:0E120200BFFF29C002C003C0049000B2E0FA92
:0E12100075F00AA4FAEE24D09000B22AF090F5
:0D121E0000B2E0FAD004D003D002709BD2E1
:03122B00098097A0
:0E122E00EF75F00AA4FFEE24D09000B32FF06D
:03123C000211C5D7
:0E123F009000B5E0FEBE2E089000B3E4F00271
:02124D0011C5C9
:0E124F008E82C002C003C004C006121F4BE511
:0C125D008224FF9207D006D004D003D0FA
:0B126900023007079000B574DF5EF054
:0A1274009000B5E0FEBE2002805598
:05127E00BE2B02804BB5
:05128300BE2D028041B8
:05128800BE4202804B94
:05128D00BE4302805089
:06129200BE44030214C675
:06129800BE46030214E84B
:06129E00BE49030214C664
:0512A400BE4C02803485
:0612A900BE4F030214D049
:0612AF00BE5003021428EA
:0512B500BE530280425F
:0612BA00BE55030214D82A
:0612C000BE58030214E019
:0312C6000214EC23
:0512C900D2080211C56E
:0512CE00D20A0211C567
:0512D300D20B0211C561
:0512D800D20D0211C55A
:0512DD00D20E0211C554
:0E12E2009000AEE0FA24FEF89000AEF0860216
:0C12F000088603188A821210500214F8BD
:0E12FC009000AEE0FA24FDF89000AEF08602FD
:0E130A00088603088604181890009DEAF0A3D8
:0E131800EBF0A3ECF090009DE0FAA3E0FBA345
:0E132600E0FC8A828B838CF0121A72AA82ABD2
:0E133400839000B3E0FBBBFF059000B3EAF02E
:0C1342002008389000B2E0FBC3EA9B508A
:0D134E002E9000B2EBC39AF09000B2E0FBCD
:0D135B008B041B9000B2EBF0BC0002801070
:0E136800758220C002C003121050D003D002C4
:0213760080E312
:051378009000B2EBF053
:05137D009000B3E0FD4B
:0E138200C00290009DE0FCA3E0FFA3E0FA8C07
:0E139000828F838AF0121E79D00260538D0482
:0E139E001DC374808CF063F08095F05044C045
:0A13AC000290009DE0F50FA3E0F5AC
:0813B60010A3E0F511740125FC
:0713BE000FFBE43510FAAC4F
:0C13C5001190009DEBF0A3EAF0A3ECF007
:0713D100850F828510838562
:0C13D80011F0121E79FAF582C002C00567
:0B13E400121050D005D002D002809300
:0613EF002008030214F8BF
:0D13F5009000B2E0FBC3EA9B40030214F835
:0C1402009000B2EBC39AF09000B2E0FA48
:0E140E008A031A9000B2EAF0BB00030214F346
:0C141C00758220C002121050D00280E641
:0E1428009000AEE0FB24FDF89000AEF08603CD
:0E143600088604088607181890009DEBF0A3A6
:0E144400ECF0A3EFF090009FE0FB247F500837
:081452009000B57443F0802006
:0D145A00EB249F50089000B57450F08013F3
:0D146700EB24BF50089000B57449F08006DA
:061474009000B57458F071
:0E147A009000B5E0FBF582C003121050D003C5
:0E14880075823AC003121050D003758230C036
:0E14960003121050D003758278C0031210505C
:0714A400D003BB4902800FD9
:0514AB00BB5002800AA5
:0A14B00090009EE0FBF5821210BAD6
:0C14BA0090009DE0FBF5821210BA803219
:0A14C600D20C9000B1740AF08028E7
:0814D0009000B17408F08020C7
:0814D8009000B1740AF08018C5
:0814E0009000B17410F08010BF
:0414E800D20F800C93
:0714EC008E821210508005F2
:0514F3009000B2EAF0D8
:0C14F800300F6B9000AEE0FA24FCF8907E
:0E15040000AEF08602088603088604088606FC
:0E15120018181890009DEAF0A3EBF0A3ECF07F
:0B152000A3EEF090009D7485F0A37412
:06152B001FF0A37480F024
:0E15310090009DE0FBA3E0FCA3E0FD74012B05
:0E153F00FEE43CFF8D0290009DEEF0A3EFF065
:0E154D00A3EAF08B828C838DF0121E79FA7067
:04155B000302116A0C
:07155F008A8212105080CBBC
:0B1566009000B1E0FABA000302116A25
:081571009000BC74BBF0A374F0
:0615790000F0300D4C9063
:0E157F0000AEE0FA14F89000AEF08602EA33F7
:0E158D0095E0FBFCFE90009DEAF0A3EBF0A3BE
:0B159B00ECF0A3EEF0300C0302164051
:0E15A60090009DE0FAA3E0FBA3E0FCA3E0FEB2
:0E15B4007B007C007E0090009DEAF0A3EBF02F
:0815C200A3ECF0A3EEF080762B
:0C15CA00300E2A9000AEE0FA24FCF890ED
:0E15D60000AEF086020886030886040886062A
:0E15E40018181890009DEAF0A3EBF0A3ECF0AD
:0515F200A3EEF08049AA
:0E15F7009000AEE0FA24FEF89000AEF08602FE
:0E16050008860318EB3395E0FCFE90009DEA8A
:0C161300F0A3EBF0A3ECF0A3EEF0200C31
:0E161F002090009DE0FAA3E0FBA3E0FCA3E016
:0E162D00FE7C007E0090009DEAF0A3EBF0A38F
:05163B00ECF0A3EEF04D
:0C164000300C3E90009DE0FAA3E0FBA3FC
:0E164C00E0FCA3E0FE30E72B90009DE0FAA347
:0E165A00E0FBA3E0FCA3E0FEC3E49AFAE49BED
:0E166800FBE49CFCE49EFE90009DEAF0A3EBE8
:09167600F0A3ECF0A3EEF08002F9
:02167F00C20C9B
:08168100D2109000B1E0FC75ED
:0316890012BB751C
:04168C0013007D00CA
:0E1690009000A1E4F08C82C004C0051210DAB4
:0C169E00D005D004201032C0049000A140
:0A16AA00E0FFC4FF85128285138360
:0A16B400E0FA4207851282851383D5
:0A16BE00EFF0151274FFB5120215CB
:0116C800130E
:0816C9009000BCE512F0A3E55E
:0616D10013F0D004800CB0
:0916D7009000A1E0FF851282855C
:0316E0001383F081
:0916E3000D9000B4EDF0B210907E
:0E16EC00009DE0FFA3E0FAA3E0FEA3E0FBEF09
:0C16FA004A4E4B70919000BCE512F0A32A
:09170600E513F09000B4EDF09041
:0C170F0000B2E0FA70069000B27401F025
:0A171B0020092720082474012DFA8C
:051725009000B2E0FBA2
:0D172A00C3EA9B5011758220C002C003125B
:091737001050D003D0021B80EA1F
:051740009000B2EBF087
:0A174500300C1275822D1210509026
:0B174F0000B2E0FA149000B2F0802F0E
:0C175A009000B4E0FA6028300A1275829A
:0B1766002B1210509000B2E0FA14901B
:0517710000B2F080133E
:0A177600300B107582201210509005
:0917800000B2E0FA149000B2F08E
:0917890020082F9000B4E0FA9052
:0417920000B2E0FBC6
:0E1796008B041B9000B2EBF0C3EA9C5036307F
:0617A40009047C30800204
:0217AA007C20A1
:0E17AC008C82C002C003121050D003D0028005
:0117BA00DB53
:0E17BB009000B2E0FA9000B4E0FCC39A50092E
:0917C9009000B2EAC39CF0800C10
:0717D2009000B2E4F0800575
:0517D9009000B2EBF0EE
:0D17DE009000BCE0FAA3E0FB9000B4E0FC3A
:0A17EB008C061CEE6040B2102010C6
:0617F500150ABA00010B09
:0E17FB008A828B83E0FEC4540FFE9000A1F0A2
:02180900800E4F
:0E180B008A828B83E0FE53060F9000A1EEF060
:0E1819009000A1E0FEF582C002C003C00412E0
:0A1827001098D004D003D00280BA5C
:0618310020080302116A09
:051837009000B2E0FA90
:09183C008A031AEB700302116A21
:0C184500758220C002121050D00280EB0F
:081851008D8212105002116A91
:0C1859009000A2E0FAA3E08A82F583224E
:0B1F85003C4E4F20464C4F41543E00A4
:0B186500E5829000C0F0301102C29438
:091870009000C0E0FA7B007C004E
:0E1879008A057E009000CF7488F0A37413F0EF
:0E1887008D828E83C002C003C004121A52ADBF
:0E18950082AE83D004D003D002C3EB9DEC647E
:0E18A300808EF063F08095F050070BBB00C8FC
:0318B1000C80C5E3
:0518B400301102D29486
:0118B900220C
:0C18BA00E582FA901F9093FAC4540FFBD3
:0218C6007C00A4
:0D18C800C3EC9B50528CF005F074018002BF
:0218D50025E00C
:0C18D700D5F0FBFD5A6016D2117582039B
:0E18E300C002C003C004121865D004D003D0A8
:0318F1000280145E
:0C18F400D211758201C002C003C00412B2
:081900001865D004D003D002E9
:0C190800C211758201C002C003C00412AD
:0B1914001865D004D003D0020C80A99D
:0C191F00C211758203C002C003121865DB
:06192B00D003D0028095FC
:0A193100121AC5900014121AC6C263
:0A193B0013900014121AE3D29490E6
:0519450018BA02196B45
:0C194A00E5829000C1F09000C1E0FA744A
:081956006AC0E07419C0E090C2
:0C195E0000BEE0C0E0A3E0C0E08A8222EE
:01196A00225A
:0E196B00AA83E5829000C2F0A3EAF09000C2C9
:0E197900E0FAA3E0FB9000BEEAF0A3EBF02240
:0E198700E5829000C4F09000C4E025E0FA2450
:0A199500E4F582E43400F583E0FA83
:0C199F00A3E0FB7C808A828B838CF0220A
:031F9000002148E5
:091F93004E6F206572726F72003E
:0E1F9C0049324320646576696365206E6F7478
:091FAA002070726573656E74000D
:0E1FB300493243206465766963652064696481
:091FC100206E6F742061636B0057
:021FD500931F58
:021FD7009C1F4D
:021FD900B31F34
:0200BD00C2126D
:0E19AB00C2AF9000C5E0FAA3E0FBA3E0FCA3EE
:0E19B900E0FD9000C9EAF0A3EBF0A3ECF0A370
:0C19C700EDF0D2AF8A828B838CF0ED2211
:0E19D300C0E0C082C083C0D075D0009000C5B7
:0E19E100E02401F0A3E03400F0A3E03400F0B5
:0E19EF00A3E03400F0C2CFD0D0D083D082D09D
:0219FD00E032D6
:0419FF00301201227F
:0E1A030075C900C2C9C2C8C2CDC2CCC2CBC216
:0D1A1100CAC2CF120B7CE433FABA010E906A
:0D1A1E0000CD74F3F09000CE74FFF0800C4A
:0C1A2B009000CD74F9F09000CE74FFF034
:0E1A37009000CDE0FA8ACD9000CEE0FB8BCC83
:0C1A45008ACB8BCAD2CAD2AFD2E8D21230
:011A51002272
:0E1A5200AA83AB828BF09000CFE0A4F8A9F03D
:0E1A60008AF0E0A429F98BF0A3E0A429F58315
:041A6E008882222226
:0E1A7200AAF0AB83E5829000D1F0A3EBF0A3C5
:0E1A8000EAF07A007B009000D1E0FCA3E0FDCC
:031A8E00A3E0FED4
:0E1A91008C828D838EF0121E79FFA3AC82AD85
:0E1A9F00839000D1ECF0A3EDF0A3EEF0EF6029
:081AAD00070ABA00DF0B80DC20
:0E1AB5009000D1ECF0A3EDF0A3EEF08A828B4E
:021AC30083227C
:011AC50022FE
:011AC60022FD
:0E1AC700AA83E5829000D4F0A3EAF09000D448
:0C1AD500E0FAA3E0FBD2148A828B8302AB
:021AE1001B01E7
:0E1AE300AA83E5829000D6F0A3EAF09000D628
:0A1AF100E0FAA3E0FBA21392148AAE
:061AFB00828B83021B0137
:0E1B0100AA83E5829000D8F0A3EAF09000D805
:091B0F00E0FAA3E0FB30E701223B
:0E1B1800C374439A74808BF063F08095F05094
:021B260001229A
:0D1B2800EA240983C0E0EA244783C0E022DC
:021B3500BDC22F
:021B3700C7CC19
:021B3900D1D603
:021B3B00DBE0ED
:021B3D00888896
:021B3F00888894
:021B4100888892
:021B4300888890
:021B4500E5EACF
:021B4700EFF4B9
:021B4900F9FEA3
:021B4B0003088D
:021B4D00888886
:021B4F00888884
:021B5100888882
:021B5300888880
:021B55000D126F
:021B5700171C59
:021B5900212643
:021B5B002B302D
:021B5D00888876
:021B5F00888874
:021B6100888872
:021B6300888870
:021B6500353A0F
:021B67003F44F9
:021B6900494EE3
:021B6B005358CD
:021B6D00888866
:021B6F00888864
:021B7100888862
:021B7300888860
:021B75005D68A9
:021B7700737E7B
:021B79001B1B34
:021B7B001B1B32
:021B7D001B1B30
:021B7F001B1B2E
:021B81001C1C2A
:021B83001C1C28
:021B85001C1C26
:021B87001C1C24
:021B89001B1B24
:021B8B001B1B22
:021B8D001B1B20
:021B8F001C1C1C
:021B91001C1C1A
:021B93001C1C18
:021B95001C1C16
:021B97001C1C14
:021B99001C1C12
:021B9B001C1C10
:021B9D001C1C0E
:021B9F001C1C0C
:021BA1001C1C0A
:021BA3001C1C08
:021BA5001C1C06
:021BA7001C1C04
:021BA9001C1C02
:021BAB001C1C00
:021BAD001C1CFE
:021BAF001C1CFC
:021BB1001C1CFA
:021BB3001C1CF8
:021BB5001C1CF6
:021BB7001C1CF4
:021BB9001C1CF2
:021BBB001C1CF0
:051BBD00A21492802239
:051BC200A21492812233
:051BC700A2149282222D
:051BCC00A21492832227
:051BD100A21492842221
:051BD600A2149285221B
:051BDB00A21492862215
:051BE000A2149287220F
:051BE500A21492902201
:051BEA00A214929122FB
:051BEF00A214929222F5
:051BF400A214929322EF
:051BF900A214929422E9
:051BFE00A214929522E3
:051C0300A214929622DC
:051C0800A214929722D6
:051C0D00A21492A022C8
:051C1200A21492A122C2
:051C1700A21492A222BC
:051C1C00A21492A322B6
:051C2100A21492A422B0
:051C2600A21492A522AA
:051C2B00A21492A622A4
:051C3000A21492A7229E
:051C3500A21492B02290
:051C3A00A21492B1228A
:051C3F00A21492B22284
:051C4400A21492B3227E
:051C4900A21492B42278
:051C4E00A21492B52272
:051C5300A21492B6226C
:051C5800A21492B72266
:071C5D0030140443A1012231
:041C640053A1FE2268
:071C680030140443A1022225
:041C6F0053A1FD225E
:071C730030140443A1042218
:041C7A0053A1FB2255
:071C7E0030140443A1082209
:031C850053A1F771
:011C88002239
:0E1C8900AA83E5829000DAF0A3EAF09000DA78
:0B1C9700E0FAA3E0FB30E703021E654B
:0E1CA200C374439A74808BF063F08095F05009
:041CB00003021E65A8
:0D1CB400EA240983C0E0EA244783C0E0224F
:021CC100495088
:021CC300575E6A
:021CC500656C4C
:021CC700737A2E
:021CC90065654F
:021CCB0065654D
:021CCD0065654B
:021CCF00656549
:021CD100818808
:021CD3008F96EA
:021CD5009DA4CC
:021CD700ABB2AE
:021CD90065653F
:021CDB0065653D
:021CDD0065653B
:021CDF00656539
:021CE100B9C088
:021CE300C7CE6A
:021CE500D5DC4C
:021CE700E3EA2E
:021CE90065652F
:021CEB0065652D
:021CED0065652B
:021CEF00656529
:021CF100F1F808
:021CF300FF06EA
:021CF5000D14CC
:021CF7001B22AE
:021CF90065651F
:021CFB0065651D
:021CFD0065651B
:021CFF00656519
:021D010029387F
:021D0300475641
:021D05001D1DA2
:021D07001D1DA0
:021D09001D1D9E
:021D0B001D1D9C
:021D0D001E1E98
:021D0F001E1E96
:021D11001E1E94
:021D13001E1E92
:021D15001D1D92
:021D17001D1D90
:021D19001D1D8E
:021D1B001D1D8C
:021D1D001E1E88
:021D1F001E1E86
:021D21001E1E84
:021D23001E1E82
:021D25001D1D82
:021D27001D1D80
:021D29001D1D7E
:021D2B001D1D7C
:021D2D001E1E78
:021D2F001E1E76
:021D31001E1E74
:021D33001E1E72
:021D35001D1D72
:021D37001D1E6F
:021D39001E1E6C
:021D3B001E1E6A
:021D3D001E1E68
:021D3F001E1E66
:021D41001E1E64
:021D43001E1E62
:021D45001E1E60
:021D47001E1E5E
:071D4900E4A2803324FF2215
:071D5000E4A2813324FF220D
:071D5700E4A2823324FF2205
:071D5E00E4A2833324FF22FD
:071D6500E4A2843324FF22F5
:071D6C00E4A2853324FF22ED
:071D7300E4A2863324FF22E5
:071D7A00E4A2873324FF22DD
:071D8100E4A2903324FF22CD
:071D8800E4A2913324FF22C5
:071D8F00E4A2923324FF22BD
:071D9600E4A2933324FF22B5
:071D9D00E4A2943324FF22AD
:071DA400E4A2953324FF22A5
:071DAB00E4A2963324FF229D
:071DB200E4A2973324FF2295
:071DB900E4A2A03324FF2285
:071DC000E4A2A13324FF227D
:071DC700E4A2A23324FF2275
:071DCE00E4A2A33324FF226D
:071DD500E4A2A43324FF2265
:071DDC00E4A2A53324FF225D
:071DE300E4A2A63324FF2255
:071DEA00E4A2A73324FF224D
:071DF100E4A2B03324FF223D
:071DF800E4A2B13324FF2235
:071DFF00E4A2B23324FF222D
:071E0600E4A2B33324FF2224
:071E0D00E4A2B43324FF221C
:071E1400E4A2B53324FF2214
:071E1B00E4A2B63324FF220C
:071E2200E4A2B73324FF2204
:091E2900E5A130E0047A01800219
:021E32007A0034
:041E3400EA24FF227B
:091E3800E5A130E1047A01800209
:021E41007A0025
:041E4300EA24FF226C
:091E4700E5A130E2047A018002F9
:021E50007A0016
:041E5200EA24FF225D
:091E5600E5A130E3047A018002E9
:021E5F007A0007
:041E6100EA24FF224E
:041E6500E424FF2250
:03003F00758122A6
:0A004200121E69E58260030200C28D
:071E6900758E0090000022BD
:091E700012003E121931C2A62233
:081FCA00240025002600270079
:0E1E790020F71430F6148883A88220F507E6BF
:061E8700A8837583002210
:031E8D00E280F7F9
:031E9000E49322B6
:021E9300E0224B
:0A1E9500900001120117E424FF225F
:0D1E9F00E5829000DCF0C2A5D2A4D2A6908E
:0D1EAC0000DCE0FAC454F0FA9000DCF09085
:0E1EB90000DCE0FA74F05A428043020FEA5255
:061EC70080C2A6D2A52294
:061ECD00E5829000DDF04B
:0E1ED300121E9540FB9000DDE0FAC4540FFB98
:0E1EE10053030F8B82C002121E9FD0025302C9
:061EEF000F8A82021E9F13
:0D1EF500E5829000DEF0C2A5C2A4D2A69046
:0D1F020000DEE0FAC454F0FA9000DEF0902A
:0E1F0F0000DEE0FA74F05A428043020FEA52FC
:061F1D0080C2A6D2A5223D
:061F2300E5829000DFF0F2
:0E1F2900121E9540FB9000DFE0FAC4540FFB3F
:0E1F370053030F8B82C002121EF5D00253021C
:061F45000F8A82021EF566
:0E1F4B00E5829000E0F09000E0E0FABA61005C
:0B1F59004009EA248540047582012243
:041F64007582002260
:01003E00229F
:08006E007909E94400601A7AE7
:050076000143A201900E
:05007B001FD215A29048
:0800800000E1E405A293A315C1
:07008800A2F0A3D9F5DAF3A1
:00000001FF
